:020000040800F2
:10000000F04900204D0100082119000815110008D1
:100010001D190008C30200086D2C00080000000034
:100020000000000000000000000000007B1C000831
:10003000A30B00080000000063010008D91D0008A0
:1000400067010008670100086701000867010008F0
:1000500067010008670100086701000867010008E0
:1000600067010008670100086701000867010008D0
:10007000ED09000867010008EF09000867010008A2
:1000800067010008670100086701000867010008B0
:1000900067010008670100086701000867010008A0
:1000A0006701000867010008670100086701000890
:1000B0006701000867010008670100086701000880
:1000C0006701000867010008670100086701000870
:1000D000670100081D270008252700082D270008B4
:1000E0006701000867010008670100086701000850
:1000F0006701000867010008670100086701000840
:10010000670100086701000867010008670100082F
:10011000670100086701000867010008670100081F
:10012000670100086701000867010008670100080F
:10013000DFF80CD000F094F8004800477D33000849
:10014000F049002080F30888704700000648804787
:1001500006480047FEE7FEE7FEE7FEE7FEE7FEE7AC
:10016000FEE7FEE7FEE7FEE7011E0008310100089A
:1001700040EA01039B0703D009E008C9121F08C029
:10018000042AFAD203E011F8013B00F8013B521EA9
:10019000F9D27047D2B201E000F8012B491EFBD220
:1001A00070470022F6E710B513460A460446194682
:1001B000FFF7F0FF204610BD421E12F8013F002B52
:1001C000FBD111F8013B02F8013B002BF9D170473C
:1001D00010B5002200E0521C835C8C5CA34201D16C
:1001E000002BF8D1D8B2E1B2401A10BD034611F885
:1001F000012B00F8012B002AF9D1184670472DE990
:10020000F05F0546002092469B468846064681469A
:1002100040241BE0284641464746224600F041F86C
:1002200053465A46C01A914110D3114618462246E9
:1002300000F028F82D1A67EB01084F4622460120EE
:10024000002100F01FF817EB00094E41201EA4F119
:100250000104DFDC484631462A464346BDE8F09FAC
:10026000064C074D06E0E06840F0010394E8070003
:1002700098471034AC42F6D3FFF75EFF4C390008C4
:100280006C390008202A04DB203A00FA02F1002031
:1002900070479140C2F1200320FA03F319439040C4
:1002A0007047202A04DB203A21FA02F0002170472F
:1002B00021FA02F3D040C2F12002914008431946CE
:1002C000704700BFFEE700002DE9F0414FF0000845
:1002D0002E494968491E01EB410202EBC1022B493C
:1002E000083101EB82002AA1FFF772FF10B14FF035
:1002F000010810E025484068401E00EB400101EB7A
:10030000C0012248083000EB8100406AB0F5805FF0
:1003100001D94FF00208B8F1000F08D006E01EA086
:1003200001F00CF94FF4FA7000F03CFCF7E70026FE
:1003300028E016484068401E00EB400101EBC00178
:100340001248083000EB8100846A4FF4FF151EB993
:1003500004F5805405F58055002710E04FF48062C5
:100360002146124803F09CF84FF4806229460F485A
:1003700003F00AF904F5806405F580657F1C042FFD
:10038000ECD3761C022ED4D3BDE8F0816E2600207B
:100390007379732E696E69007379732E696E6920A3
:1003A0006572722C2073746F700D0A006E2200202B
:1003B0002DE9F04104460D46164633462A462146AD
:1003C000044801F025FA07463946024802F038FC95
:1003D000BDE8F0815621002010B5044801F04AFA2A
:1003E00004462146014802F02BFC10BD5621002096
:1003F0002DE9F04F91B007460297029F3868FE49F9
:10040000884204D04FF0FF3011B0BDE8F08F029861
:100410000079952802D06FF00100F5E70298407945
:1004200010900298008B0F90109803287ED10F989F
:10043000A0F57061823902D06FF00300E4E73D4619
:10044000B5F89ABF4FF4786205F11A01002002F066
:1004500025FF8246DA4502D06FF00400D4E7D5F8D4
:100460001E0008B90020CFE705F11A0001F03CFB9F
:1004700005F11A0000F046FDE0490880D5F81E009D
:100480000988884209D8D5F81E00DD494860DD4852
:10049000086000F035FD0020B6E7D5F81E00D84909
:1004A0004860D64804888EE054B9002104EB44002B
:1004B00000EBC402D248083000EB8200816245E0C4
:1004C000601E00EB400101EBC001CD48083000EB9D
:1004D0008100808CC0F30B09601E00EB400101EB32
:1004E000C001C748083000EB8100806A00F58050E9
:1004F000611E01EB410202EBC102C149083101EB6F
:100500008201496A014404EB440000EBC402BC4888
:10051000083000EB82008162B9F1000F16D004EBC5
:10052000440000EBC401B648083000E088E000EB6E
:100530008100806AC9F58051014404EB440000EB5E
:10054000C402AF48083000EB8200816204EB440033
:1005500000EBC40105F1220000EB8100416A04EBCD
:10056000440000EBC402A648083000EB8200416260
:1005700004EB440202EBC40305F1220202EB830206
:1005800002F1140104EB440202EBC4039C4A08325A
:1005900002EB830202F114001022FFF7E9FD04EBE5
:1005A000440202EBC40305F1220202EB830104EBD7
:1005B000440202EBC403924A083202EB8300142285
:1005C000FFF7D6FD641C8E484068A0423FF66CAF32
:1005D00000208D4908608A4842688CA1904802F04A
:1005E00005FC8F4800F0AAFF8448008800EB40011A
:1005F00001EBC0018248083000EB8100406A0090A6
:100600007E48008800EB400101EBC0017C480830C7
:1006100000EB810383487949098830F8112082A1D1
:100620007F4802F0E3FB7E4800F088FF4FF48052E1
:100630007548016871480088FFF7BAFE0120E3E6BB
:10064000109804287DD13E46D6F83E106B480088AD
:1006500000EB400202EBC0026948083000EB820068
:10066000406A81420DD1B06C67490968884208D15F
:100670006C486249098830F81100B6F84610884283
:100680000DD06FA000F05AFF4FF480525E48016811
:100690005A480088FFF78CFE6FF00500B4E6D6F8E4
:1006A0004C80A8F10208424606F15001002002F0F9
:1006B000F5FD834606F1500008F10101405C4FEA68
:1006C000002A06F1500010F8080050441FFA80FA82
:1006D000DA450DD061A000F031FF4FF480524A4856
:1006E000016846480088FFF763FE6FF007008BE65D
:1006F0001FFA88F24148008800EB400303EBC00377
:100700003F48083000EB8300806A00F580503E4B84
:100710001B68C11806F1500002F036FF3A48006825
:1007200008EB0001D6F83E00814263D333480088CD
:1007300000F00EFB78BB0020334908602F4800888A
:1007400000E031E100EB400101EBC0012C48083032
:1007500000EB8100406A00902848008800EB4001CF
:1007600001EBC0012648083000EB81032D482349E6
:10077000098830F811202CA1294802F037FB2848BD
:1007800000F0DCFE4FF480521F4801681B480088CF
:10079000FFF70EFE06E1FFE71848008800EB400176
:1007A00001EBC0011648083000EB8100406A0C9054
:1007B0001248008800EB400202EBC00210480830EB
:1007C00000EB8201142203A8FFF7D2FC0B4800883B
:1007D00000EB400202EBC0020948083000EB820047
:1007E00000F11401102208A8FFF7C2FC1F480E9068
:1007F00002483DE0AEE00000504354417800002044
:100800006E260020F8DEBC8A7C0000205246696C0F
:100810006520436F756E743D256C750D0A000000F0
:100820006E220020BA2100205246696C655B256467
:100830005D3A2573206C656E3D256C750D0A0000D0
:10084000464C656E206F72204F6666736574206536
:100850007272215265444F210D0A00004352432019
:10086000657272215265444F210D0A00311B200828
:10087000008810B900200D900AE04C48008800EB79
:10088000400101EBC0014A4800EB8100806A0D90F5
:100890000C98C0F30B09DDE90C0100F58050084409
:1008A0000D90B9F1000F04D0C9F580510D9808449E
:1008B0000D903F48083841683C480088401C814200
:1008C00001D800200D903948008800EB400202EB6F
:1008D000C002374800EB8200816A302203A802F090
:1008E00053FE32480088401C80B2304908803049AD
:1008F00008394968884201D3002085E500202D4948
:1009000008602A48008800EB400101EBC00128483C
:1009100000EB8100406A00902448008800EB400111
:1009200001EBC001224800EB810323481F490988DD
:1009300030F8112021A1274802F058FA254800F08C
:10094000FDFD4FF480521B48016818480088FFF7EE
:100950002FFD27E017480068404416490860084604
:100960000068642148431149098801EB410202EB08
:10097000C1020F4901EB8201496AB0FBF1F0034665
:1009800001900C4814A10268124802F02FFA114895
:1009900000F0D4FD4FF480520648016803480088F7
:1009A000FFF706FD02202FE500BF2DE578000020AF
:1009B000762600207C000020BA2100205246696C77
:1009C000655B25645D3A257320206C656E3D256C62
:1009D000750D0A006E2200206F66667365743D25F2
:1009E0006420256425250D0A00000000704770472B
:1009F00021B1026842F00102026004E002684FF691
:100A0000FE731A400260704701684FF6FE72114093
:100A100001600021016041608160C1604B498842F2
:100A200008D14A490839496841F00F01474A083A54
:100A300051608AE045491431884208D14349083958
:100A4000496841F0F001414A083A51607DE03F4970
:100A50002831884208D13D490839496841F470611C
:100A60003A4A083A516070E038493C31884208D12E
:100A700036490839496841F47041344A083A5160AE
:100A800063E032495031884208D130490839496819
:100A900041F470212D4A083A516056E02B496431E7
:100AA000884208D129490839496841F47001274A28
:100AB000083A516049E025497831884208D12349F4
:100AC0000839496841F07061204A083A51603CE0B9
:100AD0001F49884206D1011F096841F00F01021F1A
:100AE000116032E01A491431884208D11849091FAF
:100AF000096841F0F001164A121F116025E01449FF
:100B00002831884208D11249091F096841F47061EF
:100B10000F4A121F116018E00D493C31884208D17C
:100B20000B49091F096841F47041094A121F1160FD
:100B30000BE007495031884207D10549091F096870
:100B400041F47021024A121F1160704708000240F0
:100B5000080402401AB103680B43036002E0036813
:100B60008B430360704710B50022026847F6F073AC
:100B70009A430C6A8B6823430C6923434C692343D3
:100B80008C692343CC6923434C6A23438C6A2343F7
:100B90001A430260CB6843600B6883604B68C36094
:100BA00010BD704710B5024607E0002101E04B1C64
:100BB00099B241F270739942F9DB1300A2F101047A
:100BC000A2B2F2D110BD4FF0E0231A6900210CE06F
:100BD00008E04FF0E0231B69934203D04FF0E0237D
:100BE0001A6900E0F5E700BF491C8142F0DB70475D
:100BF00001461CE000BF00BF00BF00BF00BF00BF38
:100C000000BF00BF00BF00BF00BF00BF00BF00BFEC
:100C100000BF00BF00BF00BF00BF00BF00BF00BFDC
:100C200000BF00BF00BF00BF00BF00BF00BF0A0081
:100C3000A1F1010399B2DDD17047000030B504463F
:100C400004254FF4302000F06FF80546042D17D12D
:100C50000C48006940F002000A49086108464461F6
:100C6000006940F0400008614FF4302000F05CF86B
:100C700005460448006941F6FD71084001490861D4
:100C8000284630BD0020024004200B49C96811F0FD
:100C9000010F01D001200EE00749C96811F0040FCF
:100CA00001D0022007E00449C96811F0100F01D0FB
:100CB000032000E004207047002002400348006940
:100CC00040F08000014908617047000000200240A8
:100CD00070B504460D460426F00200F025F80646DD
:100CE000042E11D10948006940F00100074908614C
:100CF0002580F00200F018F806460448006941F625
:100D0000FE71084001490861304670BD0020024074
:100D1000024803494860034848607047230167451B
:100D200000200240AB89EFCD00B502460423FFF757
:100D3000ABFF034603E0FFF7A7FF0346521E012B5C
:100D400001D1002AF7D102B90523184600BD0000E1
:100D50002DE9F043ADF26C4D064606EB460000EB84
:100D6000C6012B4800EB8100D0F8249006EB46002A
:100D700000EBC601264800EB8100876A07F5805723
:100D8000B8464D460DF2044000F07AFC20E0B5F57F
:100D9000806F11D94FF48062414601A802F080FBB8
:100DA0004FF4806201A90DF2044000F07BFC08F5CD
:100DB0008068A5F580650BE0AAB2414601A802F063
:100DC0006FFB2A4601A90DF2044000F06BFC0025E0
:100DD000002DDCD10DF2044000F0EAFB002413E00A
:100DE00006EB460000EBC601094800EB8100143019
:100DF000015D0DF25C40005D814204D000200DF2E7
:100E00006C4DBDE8F083641C102CE9DB0120F6E793
:100E10007626002010B500F017F809480068094947
:100E200088420BD04FF478610548FFF7BAF90548BE
:100E30000349086000F064F8012010BD0020FCE7C1
:100E40006E260020F8DEBC8A30B58DB04FF4786194
:100E50002748FFF7A6F9002400253DE03022294667
:100E600001A802F01DFB23490C98884232D104EB03
:100E7000440101EBC4021E49083101EB8200142237
:100E800001A9FFF775F904EB440101EBC40218490D
:100E9000083101EB820101F11400102206A9FFF7CD
:100EA00067F904EB440000EBC4021148083000EB82
:100EB00082000A99416204EB440000EBC4010C4833
:100EC000083000EB81008562641C0B9808B10B9D13
:100ED00002E004E005F5805507488542BEDB00BF0F
:100EE0000348446014B10548014908600DB030BDA5
:100EF0006E260020311B2008FFDF1F00F8DEBC8AB1
:100F00007047000070B50646002446E004EB44003C
:100F100000EBC401254800EB8100416A04EB44006A
:100F200000EBC40206F1080000EB8200406A814237
:100F300000D037E0002516E004EB440000EBC401CC
:100F40001A4800EB81001430415D04EB440000EBD3
:100F5000C40206F1080000EB82001430405D8142BB
:100F600000D002E06D1C102DE6DB00BF102D00D07C
:100F700018E004EB440202EBC40306F1080202EBA2
:100F8000830104EB440202EBC403084A02EB830032
:100F9000FFF71EF900B105E0641C044808384068FA
:100FA000A042B3D800BF204670BD000076260020C6
:100FB0002DE9F041024600250026002000230024F0
:100FC000002791F803C00CF00F0591F803C01CF046
:100FD000100F03D091F802C04CEA050591F800C04B
:100FE000BCF1000F31D0146800202BE04FF0010C51
:100FF0000CFA00F3B1F800C00CEA03069E4220D1BF
:1010000083004FF00F0C0CFA03F7BC4305FA03FC06
:101010004CEA040491F803C0BCF1280F06D14FF04C
:10102000010C0CFA00FCC2F814C00AE091F803C0ED
:10103000BCF1480F05D14FF0010C0CFA00FCC2F8CE
:1010400010C0401C0828D1D31460B1F800C0BCF116
:10105000FF0F34DD546800202EE000F1080C4FF043
:10106000010808FA0CF3B1F800C00CEA03069E422E
:1010700021D183004FF00F0C0CFA03F7BC4305FAA3
:1010800003FC4CEA040491F803C0BCF1280F05D11D
:1010900000F1080C08FA0CF8C2F8148091F803C0AB
:1010A000BCF1480F07D100F1080C4FF0010808FA15
:1010B0000CF8C2F81080401C0828CED35460BDE85C
:1010C000F08141617047016170473EB55824684620
:1010D00000F010F8002503E01DF8050044406D1CE9
:1010E0000C2DF9DB04B95824FF2C00D185242046AF
:1010F0003EBD00000021064A00BF05E013780370E2
:10110000401C521C4B1CD9B20C29F7DB7047000065
:10111000E8F7FF1F0948C08808498988084307493C
:101120004988084305490988084305490880084655
:10113000018804A001F04AFE00BFFEE70000002085
:101140000C0000200D0A5B4846483D253034785D90
:101150000D0A00002DE9F043ADF6740D07468846F0
:101160004FF000090DF60C0000F08AFA002500246B
:1011700017E02C49601800F07DFD064628466D1CDE
:1011800003A90E54320A28466D1C0A54B5F5006FA7
:1011900006D14FF400620DF60C0000F083FA002532
:1011A000A41CBC42E5D32DB12A4603A90DF60C00C0
:1011B00000F078FA0DF60C0000F0FAF93A461AA1A0
:1011C00003A801F013FE00240BE00DF66400025D9D
:1011D0001AA101A801F00AFE01A903A8FEF7ECFF7D
:1011E000641C102CF1DB17A103A8FEF7E5FF03A890
:1011F00000F0A4F9002408E018F804100DF66400CB
:10120000005D814200D002E0641C102CF4DB00BFC2
:10121000102C04DA00200DF6740DBDE8F0830120D7
:10122000F9E700000040000846696C6553697A657B
:101230003D256420204D44353D00000025303258C6
:10124000000000000D0A000070B504460D46074876
:1012500084420AD14FF400622946054800F078FA2A
:1012600006463146024801F0EBFC70BD5043544144
:101270005621002070B504460548844207D1054830
:1012800000F098FA05462946024801F0D9FC70BDE5
:1012900050435441562100202DE9F04FA1B0804623
:1012A000444620687F49884208D020687E498842A9
:1012B00004D04FF0FF3021B0BDE8F08F20798028B6
:1012C00002D06FF00100F6E778A11DA801F08EFDB5
:1012D000A11D1DA8FEF77CFF10B16FF00200EAE728
:1012E00094F805A0208B0190BAF1000F25D1019848
:1012F000142802D06FF00300DDE7C34610220BF183
:101300001A016B48FEF734FFD846DBF82A0069491A
:1013100008600846006810B96FF00400CBE70020B1
:101320006549086065490860654908602068624948
:101330000968FFF789FF0120BDE7BAF1020F7DD1EF
:101340004746002608E05A48815D07F11A00805D93
:10135000814200D002E0761C102EF4DB00BF102E7C
:1013600008DA58A000F0EAF82068FFF783FF6FF072
:101370000500A0E7D7F82E50D7F82A000290022DDA
:101380000CD34D4902980968884207D14A48006841
:10139000291848480068801C814208D94EA000F0F6
:1013A000CDF82068FFF766FF6FF0060083E7AD1EFB
:1013B0002A4607F13201002001F070FF814607F153
:1013C0003200691C405C00021C9007F13200405D55
:1013D0001C99084480B21C901C9949450AD046A02B
:1013E00000F0ACF8206834490968FFF72DFF6FF072
:1013F000070060E720682C4988420DD1002609E0EB
:1014000007F13200805D42490978484007F1320116
:101410008855761CAE42F3D307F13202294626489E
:10142000006800F0AFF826480068284424490860A6
:101430002148006828442049086000E030E0204846
:1014400000681C490968884210DB1949194800687E
:10145000FFF780FE40B92FA000F070F82068FFF77A
:1014600009FF6FF0080026E7002024E71248006813
:10147000642148430F49096890FBF1F0034600904E
:101480000D482AA1026803A801F0B0FC03A800F0EF
:1014900055F8206808490968FFF7D6FE02200AE7D8
:1014A00000BF08E7464F544150435441300000000C
:1014B0008800002030000020380000203C00002080
:1014C000340000204D4435204D6F64696679215207
:1014D00065444F210D0A00004C656E677468206FEB
:1014E00072204F6666736574206572726F72215246
:1014F00065444F210D0A0000436865636B20435229
:1015000043206572726F72215265444F210D0A00AB
:1015100029000020436865636B204D4435206572C7
:10152000726F72215265444F210D0A004842443DBA
:10153000256420256425250D0A00000070B50546A8
:101540002C460A20FFF73FFB0BA001F03FFC0BE00D
:1015500021780B4801F0D9F900BF4021084801F07B
:1015600007F90028F9D0641C20780028F0D10A205F
:10157000FFF729FB70BD00005B4941505D00000092
:10158000003801402DE9F04104460D46164600277B
:1015900014F0010F02D00020BDE8F081AAB2034987
:1015A0006018314601F0E0FB0120F5E7004000083B
:1015B0002DE9F04190B0044620680E9060680F90CD
:1015C0002088C0F3C507382F02DAC7F1380001E0E0
:1015D000C7F17800804642462849204600F062F86C
:1015E0000026002518E004F11800E91C405C020602
:1015F00004F11800A91C405C42EA004204F1180002
:10160000691C405C42EA002004F11801495D08436E
:101610004DF82600761C2D1D0E2EE4D3694604F1EC
:10162000080000F059FC0026002521E004F1080024
:1016300010F8261050304155503830F82600C0F3CD
:10164000072204F15800691C4254503850F8260013
:10165000C0F3074204F15800A91C4254503850F816
:101660002600000E04F15801EA1C8854761C2D1D3A
:10167000042EDBD310B0BDE8F08100000A3700086B
:1016800000214160016005498160054AC260CA438A
:101690000261034AD243426170470000012345675B
:1016A00089ABCDEF2DE9F04391B004460F461546C6
:1016B0002088C0F3C509206800EBC5002168884276
:1016C00002D26068401C6060206800EBC5002060AA
:1016D000606800EB5570606033E017F8012B4846F6
:1016E00009F1010904F118010A54B9F1400F28D198
:1016F0004FF0000800261AE004F11800F11C405CCD
:10170000020604F11800B11C405C42EA004204F1F8
:101710001800711C405C42EA002004F11801895D48
:10172000084301A941F8280008F10108361DB8F165
:10173000100FE1D301A904F1080000F0CDFB4FF038
:1017400000092800A5F10105C7D111B0BDE8F0835B
:101750002DE9F04104460E4617462546322128461B
:10176000FEF71FFD0F482860802028710220687155
:101770000DA1A81D01F03AFB0C480088401C80B266
:101780000A490880E882182028831022084905F1B8
:101790001A00FEF7EDFCC5F82A60C5F82E7032205D
:1017A000BDE8F08150435441300000002C0000207F
:1017B0008800002070B5044625462C212846FEF7F7
:1017C000F0FC0D48286080202871002068710BA172
:1017D000A81D01F00BFB0A480078E882122028833C
:1017E00008A105F11A00FEF701FD002068850749F0
:1017F00008802C2070BD0000504354413000000090
:10180000290000204E554C4C000000002C00002008
:101810002DE9F04104460E461746984625465021CC
:101820002846FEF7BEFC1048286095202871042049
:1018300068710020E882362028830C4830F81600B2
:10184000A5F8460006EB460000EBC602084800EB90
:1018500082012C2205F11A00FEF78AFCC5F84C80A3
:10186000AF645020BDE8F08150435441BA210020BC
:101870007626002070B50446254622212846FEF72C
:1018800090FC0A4828609520287103206871002088
:10189000E882082028835A20A883142068834FF404
:1018A000FF10C5F81E00222070BD000050435441B7
:1018B00010B58CB016484068401E00EB400101EBAB
:1018C000C0011348083000EB8100806A00F58054A5
:1018D0000F484068401E00EB400101EBC0010C487E
:1018E000083000EB8100406A0444C4F30B00C0F5EB
:1018F000805004440748844201D30CB010BD064810
:101900000B9030222146684601F03EFE00BFF4E70E
:101910006E260020FFDF1F0012EFCDAB00BFFEE7F9
:101920007047000070B5002100230F22C4780CB36B
:10193000164C246804F4E064C4F5E064210AC1F1A3
:101940000403CA40447804FA03F184781440214324
:1019500009010F4C0678A155047804F01F050124F5
:10196000AC4005786D114FF0E02606EB8505C5F813
:10197000004109E0047804F01F050124AC40054D46
:101980000678761145F8264070BD00000CED00E0A9
:1019900000E400E080E100E002490143024A1160F6
:1019A000704700000000FA050CED00E004490978DA
:1019B000044A1170024908700121034A51717047AD
:1019C00027000020280000202000002029B1064A1E
:1019D00052690243044B5A6104E0034A526982434C
:1019E000014B5A61704700000010024029B1064ABD
:1019F00092690243044B9A6104E0034A926982436C
:101A0000014B9A61704700000010024030B5002180
:101A10000022002400232D4D6D6805F00C0121B13A
:101A2000042905D0082923D105E0294D056022E0CD
:101A3000284D05601FE0254D6D6805F47012234D9B
:101A40006D6805F48034022505EB92421CB9224DE5
:101A5000554305600BE01D4D6D6815F4003F03D044
:101A60001E4D5543056002E01A4D5543056002E0E6
:101A7000174D056000BF00BF144D6D6805F0F00103
:101A80000909174D6B5C0568DD4045600F4D6D68B9
:101A900005F4E061090A124D6B5C4568DD40856024
:101AA0000A4D6D6805F46051C90A0D4D6B5C4568BF
:101AB000DD40C560054D6D6805F44041890B094D59
:101AC0006B5CC568B5FBF3F5056130BD00100240E5
:101AD00000127A00001BB70000093D00808D5B00FA
:101AE0005000002060000020F0B58BB004460025B7
:101AF00003E0334921F815506D1C6068A842F8D8FE
:101B0000002656E006EB460101EBC60204F108018F
:101B100001EB82002BA1FEF75BFB002848D106EB0E
:101B2000460000EBC60204F1080000EB82012C2203
:101B30006846FEF71DFB374614E07A1C02EB4203B1
:101B400003EBC20304F1080202EB830107EB470237
:101B500002EBC70304F1080202EB83002C22FEF71C
:101B600007FB7F1C6068401EB842E6D86168491ECA
:101B700001EB410202EBC10204F1080101EB82001A
:101B80002C226946FEF7F4FA354606E00C49681C3B
:101B900031F8100021F815006D1C6068401EA84245
:101BA000F4D86068401E064A22F810600BB0F0BD01
:101BB000761C6068401EB042A4D800BFF6E7000063
:101BC000BA2100207379732E696E690021B10288F1
:101BD00042F04002028004E002884FF6BF731A40D0
:101BE000028070470246002013890B4201D0012079
:101BF00000E0002070470146888970478181704766
:101C000010B50022028802F441520B884C8823430D
:101C10008C882343CC8823430C8923434C8923435A
:101C20008C892343CC8923431A430280838B4FF250
:101C3000FF74234083830B8A038210BD10B50446D2
:101C400000BF02210A48FFF7CDFF0028F9D0214646
:101C50000748FFF7D3FF00BF01210548FFF7C2FF88
:101C60000028F9D00248FFF7C6FFC0B210BD00003F
:101C700000300140014608887047704710B500F0F9
:101C800001F810BD0CB500200190009030480068AC
:101C900040F480302E49086000BF2D48006800F4F1
:101CA000003000900198401C0190009818B90198EC
:101CB000B0F5A06FF1D12648006810F4003F02D0C3
:101CC0000120009001E000200090009801283ED102
:101CD0002048006840F010001E490860084600686F
:101CE00020F0030008600846006808601848406853
:101CF00017494860084640684860084640684860A0
:101D00000846406820F47C1048600846406840F46B
:101D1000302048600846006840F08070086000BFCE
:101D20000B48006810F0007FFAD00948406820F0A6
:101D30000300074948600846406840F002004860D8
:101D400000BF0348406800F00C000828F9D10CBD22
:101D5000001002400020024030B502460B461946F2
:101D6000144607E008782578A84201D0012030BD4C
:101D7000491C641C08780028F4D100BFF7E7000074
:101D800010B500200F4908600F4908600F4800781F
:101D9000122806D0342805D0562807D078280ED12E
:101DA00007E00CE00A48FFF765FA08E0FEF714FBCD
:101DB00005E00848FFF7C2FB01F0A0FA00BF00BF32
:101DC00010BD00001400002010000020270000209B
:101DD00050435441FC36000801200749C8700748A9
:101DE0000068401C05490860322804DB00200860B8
:101DF00001200149087170472000002008000020E0
:101E000010B51348006840F0010011490860084609
:101E10004068104908400E494860084600680E496D
:101E200008400B4908600846006820F480200860DC
:101E30000846406820F4FE0048604FF41F008860A8
:101E4000FFF71CFF4FF000600449086010BD000060
:101E5000001002400000FFF8FFFFF6FE08ED00E072
:101E600010B517480068401C04D015480068401C95
:101E70001349086013480078122806D034280CD083
:101E800056280BD0782818D109E00D4800680128A1
:101E900002D17820FFF78AFD0FE00EE00DE0084840
:101EA0000068042800D210BD0548007810F0010F2A
:101EB00002D005A0FFF742FB00BF00BF00BFF2E762
:101EC00014000020270000204E6F20417070210D6B
:101ED0000A00000070470000F0B505460C4628686F
:101EE0006968AA68EB6801EA020623EA01073E4333
:101EF00027683E44FE4F3E443044C60146EA5060E7
:101F0000084400EA010622EA00073E4367683E44AF
:101F1000F84F3E4433441E0346EA1353034403EA96
:101F2000000621EA03073E43A7683E44F24F3E44C1
:101F30003244560446EAD2321A4402EA030620EA40
:101F400002073E43E7683E44EC4F3E4431448E0571
:101F500046EA9121114401EA020623EA01073E43C1
:101F600027693E44E64F3E443044C60146EA50608D
:101F7000084400EA010622EA00073E4367693E443E
:101F8000E04F3E4433441E0346EA1353034403EA3E
:101F9000000621EA03073E43A7693E44DA4F3E4468
:101FA0003244560446EAD2321A4402EA030620EAD0
:101FB00002073E43E7693E44D44F3E4431448E0518
:101FC00046EA9121114401EA020623EA01073E4351
:101FD000276A3E44CE4F3E443044C60146EA506034
:101FE000084400EA010622EA00073E43676A3E44CD
:101FF000C84F3E4433441E0346EA1353034403EAE6
:10200000000621EA03073E43A76A3E44A6F524469C
:102010004F3E3244560446EAD2321A4402EA0306DC
:1020200020EA02073E43E76A3E44BB4F3E44314448
:102030008E0546EA9121114401EA020623EA0107CE
:102040003E43276B3E44B54F3E443044C60146EA0A
:102050005060084400EA010622EA00073E43676B2D
:102060003E44AF4F3E4433441E0346EA13530344F9
:1020700003EA000621EA03073E43A76B3E44A94F4B
:102080003E443244560446EAD2321A4402EA030677
:1020900020EA02073E43E76B3E44A34F3E443144EF
:1020A0008E0546EA9121114401EA030622EA03075C
:1020B0003E4367683E449D4F3E443044460146EAF5
:1020C000D060084400EA020621EA02073E43A769FD
:1020D0003E44974F3E4433445E0246EAD3530344A2
:1020E00003EA010620EA01073E43E76A3E44914FB6
:1020F0003E443244960346EA92421A4402EA0006FB
:1021000023EA00073E4327683E448B4F3E44314458
:102110000E0546EA1131114401EA030622EA0307DB
:102120003E4367693E44854F3E443044460146EA9B
:10213000D060084400EA020621EA02073E43A76A8B
:102140003E447F4F3E4433445E0246EAD353034449
:1021500003EA010620EA01073E43E76B3E44794F5C
:102160003E443244960346EA92421A4402EA00068A
:1021700023EA00073E4327693E44734F3E443144FF
:102180000E0546EA1131114401EA030622EA03076B
:102190003E43676A3E446D4F3E443044460146EA42
:1021A000D060084400EA020621EA02073E43A76B1A
:1021B0003E44674F3E4433445E0246EAD3530344F1
:1021C00003EA010620EA01073E43E7683E44614F07
:1021D0003E443244960346EA92421A4402EA00061A
:1021E00023EA00073E43276A3E445B4F3E443144A6
:1021F0000E0546EA1131114401EA030622EA0307FB
:102200003E43676B3E44554F3E443044460146EAE8
:10221000D060084400EA020621EA02073E43A768AC
:102220003E444F4F3E4433445E0246EAD353034498
:1022300003EA010620EA01073E43E7693E44494FAD
:102240003E443244960346EA92421A4402EA0006A9
:1022500023EA00073E43276B3E44434F3E4431444C
:102260000E0546EA1131114481EA02065E406769B3
:102270003E443E4F3E443044060146EA1070084456
:1022800080EA01065640276A3E44394F3E443344B3
:10229000DE0246EA5353034483EA00064E40E76AEF
:1022A0003E44344F3E443244160446EA12421A4435
:1022B00082EA03064640A76B3E442F4F3E4431441A
:1022C000CE0546EA5121114481EA02065E40676864
:1022D0003E442A4F3E443044060146EA107008440A
:1022E00080EA0106564027693E44254F3E4449E0B6
:1022F00078A46AD756B7C7E8DB702024EECEBDC1FC
:10230000AF0F7CF52AC68747134630A8019546FDD6
:10231000D8988069AFF7448BBED75C892211906B47
:10232000937198FD8E4379A62108B44962251EF663
:1023300040B340C0515A5E26AAC7B6E95D102FD6F9
:102340005314440281E6A1D8C8FBD3E7E6CDE121CE
:10235000D60737C3870DD5F4ED145A4505E9E3A92F
:10236000F8A3EFFCD9026F678A4C2A8D4239FAFF35
:1023700081F6718722619D6D0C38E5FD44EABEA4AB
:10238000A9CFDE4B3344DE0246EA5353034483EACB
:1023900000064E40E7693E449F4F3E4432441604D7
:1023A00046EA12421A4482EA03064640A76A3E44BD
:1023B0009A4F3E443144CE0546EA5121114481EA08
:1023C00002065E40676B3E44954F3E443044060132
:1023D00046EA1070084480EA0106564027683E44E9
:1023E000904F3E443344DE0246EA5353034483EAAB
:1023F00000064E40E7683E448B4F3E44324416048C
:1024000046EA12421A4482EA03064640A7693E445D
:10241000864F3E443144CE0546EA5121114481EABB
:1024200002065E40676A3E44814F3E4430440601E6
:1024300046EA1070084480EA01065640276B3E4485
:102440007C4F3E443344DE0246EA5353034483EA5E
:1024500000064E40E76B3E44774F3E44324416043C
:1024600046EA12421A4482EA03064640A7683E44FE
:10247000724F3E443144CE0546EA5121114461EA8F
:102480000306564027683E446D4F3E443044860163
:1024900046EA9060084460EA02064E40E7693E441E
:1024A000684F3E4433449E0246EA9353034463EA32
:1024B00001064640A76B3E44634F3E443244D60378
:1024C00046EA52421A4462EA00065E4067693E44A8
:1024D0005E4F3E4431444E0546EAD121114461EA43
:1024E00003065640276B3E44594F3E443044860114
:1024F00046EA9060084460EA02064E40E7683E44BF
:10250000544F3E4433449E0246EA9353034463EAE5
:1025100001064640A76A3E444F4F3E443244D6032C
:1025200046EA52421A4462EA00065E4067683E4448
:102530004A4F3E4431444E0546EAD121114461EAF6
:1025400003065640276A3E44454F3E4430448601C8
:1025500046EA9060084460EA02064E40E76B3E445B
:10256000404F3E4433449E0246EA9353034463EA99
:1025700001064640A7693E443B4F3E443244D603E1
:1025800046EA52421A4462EA00065E40676B3E44E5
:10259000364F3E4431444E0546EAD121114461EAAA
:1025A0000306564027693E44314F3E44304486017D
:1025B00046EA9060084460EA02064E40E76A3E44FC
:1025C0002C4F3E4433449E0246EA9353034463EA4D
:1025D00001064640A7683E44274F3E443244D60396
:1025E00046EA52421A4462EA00065E40676A3E4486
:1025F000224F3E4431444E0546EAD12111442E6813
:1026000006442E606E680E446E60AE681644AE607E
:10261000EE681E44EE60F0BD604BBBF670BCBFBE02
:10262000C67E9B28FA27A1EA8530EFD4051D8804D1
:1026300039D0D4D9E599DBE6F87CA21F6556ACC445
:10264000442229F497FF2A43A72394AB39A093FC93
:10265000C3595B6592CC0C8F7DF4EFFFD15D84850F
:102660004F7EA86FE0E62CFE144301A3A111084E93
:10267000827E53F735F23ABDBBD2D72A91D386EB8F
:1026800008B540F224411D4800F07FF840B31B48D4
:10269000008800901948001D008800901848C06DFF
:1026A00041F25201081A0090002115485830FEF7F7
:1026B0009FF91448007850B913491448009AFDF75F
:1026C00057FD13490098088001200E49087041F217
:1026D00052000B49C865012109485830FEF788F9B6
:1026E00008210C4800F044F8012806D1034800F006
:1026F00007F90821014800F01DF808BD0038014025
:10270000000002402000002004110020B200002040
:1027100040000020004800407047704710B5FFF7A8
:10272000AFFF10BD10B5FFF7F7FF10BD10B5FFF7F5
:10273000F4FF10BD01F40072B2F5007F00D100BFBC
:10274000CA430280704721B1828942F400528281DB
:1027500004E082894DF6FF731A40828170471AB1F6
:10276000838A0B43838202E0838A8B438382704790
:1027700002460020B1F5007F00D100BF13880B4254
:1027800001D0012000E00020704770B5024600240F
:10279000002300250020A1F510666A3E00D100BF8D
:1027A000C1F3421501F01F03012606FA03F3012DC0
:1027B00002D19689334006E0022D02D1168A3340B9
:1027C00001E0968A33400C12012606FA04F41688BA
:1027D000344013B10CB1012000E0002070BDF0B511
:1027E00003460024002600250020A1F510676A3F5B
:1027F00000D100BF1846C1F3421401F01F060127A3
:1028000007FA06F5012C01D10C3004E0022C01D1AD
:10281000103000E014301AB107682F43076002E05F
:102820000768AF430760F0BD2DE9F04786B0054665
:102830000E460024A24600BFA1460027B08900B181
:1028400000BF2F462C8A4CF6FF700440F0880443EA
:102850002C82AC894EF6F3100440B08831890843CD
:10286000718908430443AC81AC8A4FF6FF400440B1
:10287000B0890443AC8201A8FFF7C8F81F4887421B
:1028800002D1DDF810A001E0DDF80CA0A88910F459
:10289000004F08D00AEBCA0000EB0A10316849006B
:1028A000B0FBF1F807E00AEBCA0000EB0A10316850
:1028B0008900B0FBF1F86420B8FBF0F004012009B6
:1028C000642101FB1089A88910F4004F08D0322040
:1028D00000EBC900B0FBF1F000F00700044308E092
:1028E000322000EB09106421B0FBF1F000F00F0082
:1028F00004432C8106B0BDE8F08700000038014099
:1029000001468888C0F308007047C1F3080282803E
:102910007047000000B58DB001210846FFF756F85A
:102920002B48FEF771F82B4801902B48029010209D
:1029300003906420049000200590802006900020E1
:102940000790089009900A900B9001A92048FEF783
:102950000AF90E208DF8300003208DF83100022096
:102960008DF8320001208DF833000CA8FEF7DAFF55
:10297000012202211648FEF7EDF800211448FEF767
:1029800037F813481430FEF73FF812480190134807
:1029900002900020039041F2520004900020059024
:1029A0008020069000200790089009904FF4005076
:1029B0000A9000200B9001A905481430FEF7D3F8C7
:1029C000012103481430FEF713F80DB000BD0000DC
:1029D0004400024004380140562100200411002028
:1029E00000B587B0012144F20400FEF7FFFF4FF469
:1029F0000070ADF8140018208DF8170003208DF832
:102A0000160005A92E48FEF7D3FA4FF48060ADF802
:102A1000140004208DF8170003208DF8160005A976
:102A20002748FEF7C5FA4FF4E13001900020ADF8D9
:102A30000800ADF80A00ADF80C00ADF810000C204D
:102A4000ADF80E0001A91F48FFF7EEFE01211D4859
:102A5000FFF779FE4FF4E060FEF79EFF25208DF82A
:102A6000180000208DF819008DF81A0001208DF84B
:102A70001B0006A8FEF756FF40211248FFF75AFE3A
:102A8000002240F227710F48FFF7A9FE002240F212
:102A900025510C48FFF7A3FE012240F224410948CA
:102AA000FFF79DFE012240210648FFF758FE002255
:102AB00080210448FFF753FEFFF72CFF07B000BD4D
:102AC000000801400038014010B540480078122845
:102AD0001BD13FA14248FFF73FF930B93420FEF740
:102AE00065FF40A0FEF72AFD0EE042A13C48FFF73B
:102AF00033F930B95620FEF759FF42A0FEF71EFD0C
:102B000002E045A0FEF71AFD10BD304800783428D9
:102B100004D02E480078562800D0F5E730480078D9
:102B200050280BD12E484078432807D12C48807874
:102B3000542803D12A48C078412800D0E4E7284827
:102B4000007980281AD1364801882548FEF7A4FB71
:102B5000044634B933A0FEF7F1FC5620FEF726FFF9
:102B6000D2E714F1020F2EDA14F1060F2BDD30A09C
:102B7000FEF7E4FC7820FEF719FF24E018480079FE
:102B8000952820D1264801881548FDF731FC0446D8
:102B90006CB9FEF78DFEFDF797FB22A0FEF7CEFC89
:102BA0007820FEF703FF012024490870ACE714F1F8
:102BB000020F08DA14F1060F05DD1DA0FEF7BEFCBA
:102BC0007820FEF7F3FE00BF9EE7000027000020FC
:102BD000444F574E4C4F41445F415050000000005D
:102BE000B2000020444F574E4C4F41445F4150507B
:102BF0000D0A0000444F574E4C4F41445F52464926
:102C00004C455300444F574E4C4F41445F52464948
:102C10004C45530D0A0000002D2D2D2D0D0A0000EE
:102C200040000020436F6D706C6574656421000086
:102C30004941502053746F70210D0A004800002054
:102C400070B505460E4600240BE0295D0648FFF7E7
:102C50005CFE00BF40210448FFF78AFD0028F9D040
:102C6000641CB442F1DB70BD0038014000BFFEE7D8
:102C700010B586B000F036F810211848FEF723FA98
:102C80000020ADF804004FF48270ADF8060000207B
:102C9000ADF808000220ADF80A000120ADF80C00E4
:102CA0004002ADF80E000820ADF810000020ADF88D
:102CB00012000720ADF8140001A90948FEF7A0FF93
:102CC00001210748FEF782FF4FF47A70FDF790FF6D
:102CD00000F014FC0446012006B010BD00080140BD
:102CE0000030014008B501210420FEF77FFE0121DC
:102CF0000803FEF77BFE2020ADF8000003208DF8CE
:102D0000020018208DF8030069461548FEF750F9B7
:102D10008020ADF8000069461148FEF749F94020CF
:102D2000ADF8000004208DF8030069460C48FEF75A
:102D30003FF91020ADF800008DF8030069460848FF
:102D4000FEF736F91020ADF800008DF80300694653
:102D50000448FEF72DF910210248FEF7B4F908BD2A
:102D600000080140001001402DE9F04705460E46DD
:102D70009046B5F1006F02D31348854201D3BDE8F8
:102D8000F0876805400D00D0F9E7FDF7C1FF284640
:102D9000FDF754FF0746042F00D0F0E700240CE0B5
:102DA000315D601C305C01EB00201FFA80F92819AE
:102DB0004946FDF78DFFA01C84B24445F0DBFDF7CA
:102DC0007DFF00BFDBE70000000004080FB4054BE7
:102DD00010B503A9044A029800F02CF810BC5DF865
:102DE00014FB0000D9320008840000200FB4084B07
:102DF00010B504A902AA039800F01CF8044602A921
:102E0000002000F046FA204610BC5DF814FB0000DC
:102E10009332000802E008C8121F08C1002AFAD144
:102E200070477047002001E001C1121F002AFBD14A
:102E3000704700002DE9FF4F8DB00F460546002674
:102E4000DEE1252874D100246D1CF149A246A1467B
:102E500001222B78203B02FA03F0084202D00443FF
:102E60006D1CF6E728782A2810D06FF02F022878FA
:102E7000A0F13001092915D80AEB8A0102EB4101C2
:102E800044F0020400EB010A6D1CF0E757F804ABB4
:102E9000BAF1000F03DA44F40054CAF1000A44F016
:102EA00002046D1C28782E2817D115F8010F44F064
:102EB00004042A280ED06FF02F022878A0F13001E8
:102EC00009290AD809EB890102EB410100EB01094C
:102ED0006D1CF2E757F8049B6D1C28786C280FD006
:102EE00006DC4C2817D068280DD06A2814D104E0DD
:102EF000742810D07A280FD10DE044F400140AE0B1
:102F000044F4801401E044F440146978814202D111
:102F10006D1C04F580146D1C2A786E2A20D00DDCFF
:102F2000632A33D005DC002A6FD0582A12D1A2E0E0
:102F300011E0642A6AD0692A0CD167E0732A2FD085
:102F400004DC6F2A6FD0702A04D199E0752A6BD007
:102F5000782A6AD01046DDE90F129047761C4EE1C0
:102F6000C4F30250022806D003280AD0042801CF57
:102F70000AD0066043E101CF4FEAE671C0E9006183
:102F80003DE101CF06803AE1067038E117F8040B05
:102F90008DF8000000208DF80100EB46012003E0D1
:102FA00057F804BB4FF0FF3061074FF0000102D427
:102FB0000DE008F10101884649450FDA8045F8DB4C
:102FC0001BF808100029F4D108E008F10101884637
:102FD0008142FADB1BF808100029F6D1DDE90F2346
:102FE000AAEB08008146214600F03BF9304400EB93
:102FF000080604E0DDE90F121BF8010B9047B8F159
:103000000108F7D221464846F4E0FDE00A21C4F366
:1030100002534FF0000B0891022B07D001CFC117CC
:10302000032B09D00AE034E023E024E0FF1D27F061
:103030000707F7E8020105E000B2C117042B01D130
:1030400040B2C117002907DA4FF0000CD0EB0C009A
:103050006CEB01012D2302E0230504D52B238DF811
:103060002430012303E0E30701D02023F7E798464B
:1030700050E00A210EE010204FF0000B08900CE009
:1030800010214FF0000B44F004044FF008090891A0
:1030900003E008214FF0000B0891C4F30253022B08
:1030A00004D001CF0021032B06D006E0FF1D27F03E
:1030B0000707F7E8020103E080B2042B00D1C0B299
:1030C0004FF00008230725D5702A2AD0DDF820C04C
:1030D0008CF0100C5CEA0B0C09D150EA010306D00D
:1030E00030238DF824308DF8252002239846DDF812
:1030F00020C08CF0080C5CEA0B0C0BD150EA0103E9
:1031000001D1630706D530238DF824304FF0010834
:10311000A9F10109582A09D03EA20B9208AA0A92E5
:1031200011E040238DF824300123DFE73EA2F4E7CD
:103130005B46089AFDF763F80B9B9B5C0A9AA2F129
:1031400001020A92137050EA0102F1D10A98ADEB24
:10315000000000F1200B600702D524F4803401E068
:103160004FF00109D94502DDA9EB0B0000E000207A
:1031700000EB0B0141440890AAEB010AE00306D4DE
:10318000DDE90F232146504600F06BF8064400208D
:1031900008E009A911F80900DDE90F129047761C33
:1031A00009F1010081464045F3DBE0030CD5DDE980
:1031B0000F232146504600F054F8064404E0DDE9B0
:1031C0000F1230209047761C0899481E089000295D
:1031D000F5DC08E00A980A990078491C0A91DDE9B3
:1031E0000F129047761CBBF10001ABF1010BF1DC33
:1031F00021465046DDE90F2300F020F806446D1CFF
:10320000287800287FF41DAE11B03046BDE8F08F5D
:1032100009280100303132333435363738396162AC
:103220006364656600000000303132333435363770
:103230003839414243444546000000002DE9F04141
:10324000044600251E461746880405D406E0394684
:103250002020B04705F10105641EF8D52846BDE8D9
:10326000F0812DE9F041044600251E469046C80332
:1032700001D5302700E02027880405D506E0414627
:103280003846B04705F10105641EF8D52846BDE86B
:10329000F0810A68531C0B6010707047F0B5074648
:1032A0000C461546002606E014F8011B384600F0CF
:1032B00007F80746761CAE42F6D33846F0BD00004C
:1032C000024682EA0100C0B2024B33F8100080EAE5
:1032D000222070474A37000870B504460D46E1B217
:1032E0000548FFF712FB00BF40210348FFF740FAF3
:1032F0000028F9D0204670BD0038014010B50248C2
:1033000000F004F810BD00000040000810B50446AD
:10331000206814490840B0F1005F18D1002240F243
:1033200024411148FFF75BFA002240210E48FFF7C5
:1033300016FA00204FF0E021086160680B49086030
:103340002068FCF7FFFE09480068804708E006E0B7
:1033500007A0FEF7F3F84FF47A70FDF723FCF7E7C8
:1033600010BD00000000FE2F003801404400002086
:103370004E6F204170700D0A00000000FFF730FB17
:10338000304800686422B0FBF2F1B1F1807F01D3D4
:1033900001201DE021F07F40401E4FF0E0225061EF
:1033A00050170F22002807DA13071D0E264B00F0D6
:1033B0000F04241F1D5503E013071C0E234B1C5440
:1033C00000BF00204FF0E022906107201061002034
:1033D00008B100BFFEE7FFF74BFCFDF71BFDFDF753
:1033E00074FE1B4908701B480021016081808171B7
:1033F0001220FEF7DBFA24E01648007848B1FFF708
:1034000063FB00201349087041F252011248FCF797
:10341000C8FE1048407920B100200E494871FEF7DF
:10342000AFFC0C48C07820B100200A49C870FEF7F4
:1034300051FD0848007920B1002006490871FEF7C7
:103440000FFDD9E76400002018ED00E000E400E083
:103450002900002020000020B200002010B5044602
:10346000240300F0EBF800F087F810210B48FDF77B
:1034700028FE2020FEF7E2FBC4F30740FEF7DEFB48
:10348000C4F30720FEF7DAFBE0B2FEF7D7FB10210A
:103490000248FDF718FE00F06FF810BD000801406B
:1034A0002DE9F04105460C46174610211248FDF75C
:1034B00008FE0B20FEF7C2FBC4F30740FEF7BEFB7D
:1034C000C4F30720FEF7BAFBE0B2FEF7B7FBFF201C
:1034D000FEF7B4FB2870002605E0FF20FEF7AEFBE8
:1034E000A855701C86B2BE42F7DB10210248FDF7DA
:1034F000EAFDBDE8F0810000000801402DE9F0413F
:10350000002400250026002710210F48FDF7D9FDD3
:103510009F20FEF793FBFF20FEF790FB0546FF2060
:10352000FEF78CFB0646FF20FEF788FB07461021BE
:103530000548FDF7C8FD280440EA062040EA0704D4
:103540002046BDE8F08100000008014010B50024CD
:1035500010210848FDF7B5FD0520FEF76FFBFF20A1
:10356000FEF76CFB044610210248FDF7ACFD204637
:1035700010BD00000008014010B500BFFFF7E6FFD6
:1035800010F0010FFAD110BD2DE9F04781460F462A
:1035900016464FEA1738C7F30B0ACAF58054A642FD
:1035A00000DC344644E04FEA08314FF480522248B0
:1035B000FFF776FF002508E00AEB05001E49085CCE
:1035C000FF2800D003E0681C85B2A542F4DB00BFF1
:1035D000A54216DA4046FFF741FF002507E019F83B
:1035E000050005EB0A01144A5054681C85B2A54237
:1035F000F5DB4FEA08314FF480520F4800F02EF807
:1036000004E022463946484600F028F8A64200D198
:103610000FE008F101084FF0000AA1442744301BD5
:1036200086B2B6F5805F02DD4FF4805400E0344688
:10363000B9E700BFBDE8F087EE35002010B51021D6
:103640000548FDF73EFD0620FEF7F8FA1021024876
:10365000FDF739FD10BD0000000801402DE9F041E3
:1036600007460E461446F0B2C0F58075AC4200DC49
:10367000254612E02A463146384600F013F8AC429F
:1036800000D10BE02F442E44601B84B2B4F5807F40
:1036900002DD4FF4807500E02546EBE700BFBDE892
:1036A000F08100002DE9F04106460C461746FFF771
:1036B000C5FF10211048FDF704FD0220FEF7BEFAF9
:1036C000C4F30740FEF7BAFAC4F30720FEF7B6FAD0
:1036D000E0B2FEF7B3FA002504E0705DFEF7AEFA43
:1036E000681C85B2BD42F8DB10210348FDF7EBFCF6
:1036F000FFF742FFBDE8F0810008014048532D4923
:1037000041502D563130350D0A0080000000000078
:1037100000000000000000000000000000000000A9
:103720000000000000000000000000000000000099
:103730000000000000000000000000000000000089
:10374000000000000000000000000000C1C081C1B6
:10375000400101C3C003800241C201C6C006800708
:1037600041C70005C1C581C4400401CCC00C800D17
:1037700041CD000FC1CF81CE400E000AC1CA81CB1E
:10378000400B01C9C009800841C801D8C018801980
:1037900041D9001BC1DB81DA401A001EC1DE81DF86
:1037A000401F01DDC01D801C41DC0014C1D481D547
:1037B000401501D7C017801641D601D2C012801320
:1037C00041D30011C1D181D0401001F0C03080310F
:1037D00041F10033C1F381F240320036C1F681F786
:1037E000403701F5C035803441F4003CC1FC81FD17
:1037F000403D01FFC03F803E41FE01FAC03A803BA0
:1038000041FB0039C1F981F840380028C1E881E95D
:10381000402901EBC02B802A41EA01EEC02E802F07
:1038200041EF002DC1ED81EC402C01E4C024802546
:1038300041E50027C1E781E640260022C1E281E39D
:10384000402301E1C021802041E001A0C0608061EF
:1038500041A10063C1A381A240620066C1A681A705
:10386000406701A5C065806441A4006CC1AC81AD16
:10387000406D01AFC06F806E41AE01AAC06A806B1F
:1038800041AB0069C1A981A840680078C1B881B97D
:10389000407901BBC07B807A41BA01BEC07E807F87
:1038A00041BF007DC1BD81BC407C01B4C074807546
:1038B00041B50077C1B781B640760072C1B281B31D
:1038C000407301B1C071807041B00050C1908191CE
:1038D00040510193C053805241920196C056805787
:1038E00041970055C19581944054019CC05C805D16
:1038F000419D005FC19F819E405E005AC19A819B9D
:10390000405B0199C059805841980188C04880495E
:103910004189004BC18B818A404A004EC18E818F04
:10392000404F018DC04D804C418C0044C184818545
:1039300040450187C047804641860182C04280439E
:1039400041830041C1818180404000006C39000802
:103950000000002088000000142E0008F439000840
:103960008800002068490000242E000800000000A4
:103970000000000000000000000000000000000047
:103980000000000000000000000000000000000037
:103990000000000000000000000000000000000027
:1039A0000000000000000000000000000000000017
:1039B0000000000000000000000000000000000007
:1039C00001020304010203040607080902040608B1
:1039D00000366E0100000000000000000102030438
:1039E00006070809000000000000000000000000B9
:0439F00000000000D3
:0400000508000131BD
:00000001FF
